:020000040800F2
:1000000050130020010100082D2F00082D290008A1
:10001000292F0008130200083138000800000000F2
:10002000000000000000000000000000F12F0008A8
:100030003B03000800000000312F00086130000879
:100040001B0100081B0100081B0100081B01000820
:100050001B0100081B0100081B0100081B01000810
:100060001B0100081B0100081B0100081B01000800
:100070001B0100081B0100081B0100081B010008F0
:100080001B0100081B0100081B0100087137000854
:10009000D93700081B010008190200081B010008DD
:1000A0001B0100081B0100081B0100081B010008C0
:1000B0001B0100081B010008113100081B0100088A
:1000C0001B0100081B0100081B0100081B010008A0
:1000D0001B010008F53600081B0100083537000831
:1000E0001B0100081B0100081B010008DFF80CD0F1
:1000F00000F052F8004800471D510008501300203E
:100100000648804706480047FEE7FEE7FEE7FEE7B1
:10011000FEE7FEE7FEE7FEE7FEE7FEE70F31000839
:10012000ED00000840EA01039B0703D009E008C97D
:10013000121F08C0042AFAD203E011F8013B00F8AC
:10014000013B521EF9D27047D2B201E000F8012BF8
:10015000491EFBD270470022F6E710B513460A4647
:1001600004461946FFF7F0FF204610BD30B50B4698
:10017000014600202022012409E021FA02F59D42D7
:1001800005D303FA02F5491B04FA02F52844151EAB
:10019000A2F10102F1DC30BD064C074D06E0E0683B
:1001A00040F0010394E8070098471034AC42F6D3BE
:1001B000FFF7A0FF2C5E00084C5E000870B58C189D
:1001C00010F8015B15F0070301D110F8013B2A116B
:1001D00006D110F8012B03E010F8016B01F8016B58
:1001E0005B1EF9D12B0705D40023521E0DD401F854
:1001F000013BFAE710F8013BCB1A921C03E013F81D
:10020000015B01F8015B521EF9D5A142D8D3002051
:1002100070BD00BFFEE7000010B5154800684069DA
:1002200000F4007060B1124800688069C0F34000BB
:1002300010B1012003F004FD01200D490968C860D8
:100240000B480068406900F4806068B108480068A5
:100250008069C0F3800018B1002003F017FD00BFD3
:100260000120034909680861014800F0ABFA10BD9C
:10027000700100202DE9F04104460D4617461E4648
:10028000ECB10020207220606060B5F5006F03D3F0
:1002900004202072656002E000202072256006B113
:1002A00027B90020A0720220607208E0002060726E
:1002B000A6723246394604F10B00FFF733FFBDE862
:1002C000F0812DE9F04104460D4617461E46ECB17B
:1002D0000020207220606060B5F5006F03D3042019
:1002E0002072656002E000202072256006B127B907
:1002F0000020A0720220607208E000206072A672E6
:100300003246394604F10B00FFF70CFFBDE8F081DF
:100310002DE9F04107460C461546264616B1002148
:100320002846B047BDE8F08170B506460C46154634
:10033000E9B2E0B204F0E6FD70BD704772B600BFEE
:10034000FEE700000246002112E001EB410000EB55
:10035000C1000E4B03EB00100078904206D101EB78
:10036000410000EBC10003EB00107047481CC1B214
:10037000022909D201EB410000EBC100034B03EB62
:1003800000100078FF28E0D10020EEE79004002064
:1003900010B5024692F82030012B01D0022B06D175
:1003A00010684069084314686061002010BD506AFD
:1003B00040F4802050620120F8E7F0B504460D4675
:1003C0001E4694F8207020688368A86800B900E091
:1003D00000BF012F01D0022F7CD103F0806030B923
:1003E00003F0006018B903F08050002873D0C3F305
:1003F0000161022905D9606A40F4000060620120B1
:10040000F0BD012088403060A86860B9B5F800C030
:10041000E86840EA4C5C206800F5C07000EB011011
:10042000C0F800C00FE0D5E901C040EACC00D5F823
:100430000CC040EA0C00D4F800C00CF5C07C0CEBFA
:10044000011CCCF80000D5F810C0206800F5C07081
:1004500000EB0110C0F804C0287D01280ED12068EF
:1004600000F5C07000EB0110406840F4807C20680B
:1004700000F5C07000EB0110C0F804C0D079000690
:1004800092F806C040EA0C4092F805C040EA0C2CF5
:1004900010794CEA000C206800F5C07000EB0110E8
:1004A000C0F80CC0D078000692F802C040EA0C40B8
:1004B00092F801C040EA0C2092F800C040EA0C001B
:1004C000D4F800C00CF5C07C0CEB011CCCF8080083
:1004D000206801E016E00FE000F5C07000EB0110AD
:1004E000006840F0010C206800F5C07000EB0110BE
:1004F000C0F800C0002083E7606A40F4001060622A
:1005000001207DE7606A40F480206062012077E787
:10051000F0B504460A46216894F82050012D01D018
:10052000022D74D1D1F8000240F00100C1F80002A0
:10053000107D00F01F06012000FA06F3D1F81C021E
:100540009843C1F81C02D069C8B9D1F80C0298438D
:10055000C1F80C02908880B2968940EA064601F5FF
:100560001070576940F83760108880B2168940EAE9
:10057000064601F51070576900EBC7004660D06968
:10058000012819D1D1F80C021843C1F80C02908847
:1005900080B2168840EA064601F51070576940F8A7
:1005A0003760908980B2168940EA064601F51070DE
:1005B000576900EBC7004660906928B9D1F804027A
:1005C0009843C1F8040204E0D1F804021843C1F8CA
:1005D0000402106928B9D1F814029843C1F8140232
:1005E00004E0D1F814021843C1F81402106A01287B
:1005F00004D1D1F81C021843C1F81C02D1F8000242
:1006000020F00100C1F800020020F0BDFFE7606AA1
:1006100040F4802060620120F7E710B504460CB971
:10062000012010BD204600F07CFB204600F0BEFA01
:100630002068006840F40040216808600020606283
:1006400084F8200000BFECE7704770B5044694F8CA
:100650002050012D01D0022D7DD151B92068C068F4
:1006600000F0030080B9606A40F40010606201206D
:1006700070BD2068006900F0030028B9606A40F48A
:10068000001060620120F3E7206800F5D87000EBED
:100690000110006800F004009060906840B9206884
:1006A00000F5D87000EB01100068400D106007E005
:1006B000206800F5D87000EB01100068C008506099
:1006C000206800F5D87000EB0110006800F002000F
:1006D000D060206800F5D87000EB0110406800F091
:1006E0000F001061206800F5D87000EB0110406821
:1006F00000F47F40000A9061206800F5D87000EB9C
:1007000001104068000C5061206800F5D87000EBC3
:10071000011080681870206800F5D87000EB011097
:10072000806800F47F40000A5870206800F5D87097
:1007300000EB0110806800F47F00000C98702068C6
:1007400000F5D87000EB01108068000ED8702068AA
:1007500000F5D87000E02FE000EB0110C0681871C0
:10076000206800F5D87000EB0110C06800F47F40ED
:10077000000A5871206800F5D87000EB0110C068BD
:1007800000F47F00000C9871206800F5D87000EB31
:100790000110C068000ED87131B92068C06840F0FF
:1007A00020002668F06005E02068006940F0200025
:1007B0002668306100205BE7606A40F48020606258
:1007C000012055E72DE9F05F0446002520684669C1
:1007D0002068D0F80490206887682068D0F80CA0C2
:1007E0002068D0F810B02068D0F8188006F001001A
:1007F000002855D007F00100C0B1012021688860B1
:1008000007F0020018B1204600F0C1FA0EE007F030
:10081000040010B145F4006508E007F0080010B1CD
:1008200045F4805502E0204600F0B0FA07F48070ED
:10083000C8B14FF480702168886007F4007018B167
:10084000204600F0A6FA0EE007F4806010B145F4EF
:10085000005508E007F4006010B145F4804502E05F
:10086000204600F095FA07F48030C8B14FF480308C
:100870002168886007F4003018B1204600F08BFA38
:100880000EE007F4802010B145F4004508E007F4BD
:10089000002010B145F4803502E0204600F07AFADD
:1008A00006F0080038B10AF0100020B145F40075D8
:1008B00010202168C86006F0040040B10AF008006A
:1008C00028B108202168C860204600F025FA06F00B
:1008D000020038B12068C06800F0030010B1204663
:1008E00000F01BFA06F0400038B10BF0100020B108
:1008F00045F4806510202168086106F0200040B1B1
:100900000BF0080028B1082021680861204600F09B
:1009100005FA06F0100038B12068006900F0030005
:1009200010B1204600F0FBF906F4003040B109F0A8
:10093000100028B1102021684860204600F0F0F92E
:1009400006F4803040B109F0080028B10820216881
:100950004860204600F020FA06F4004088B309F011
:10096000040078B306F4807020B108F0010008B1EB
:1009700045F0010506F4007020B108F0020008B14E
:1009800045F0020506F4806020B108F0040008B1CB
:1009900045F0040506F40060A0B108F0700088B1CD
:1009A00008F07000402817D006DC10280BD0202853
:1009B0000CD0302819D10CE0502810D0602814D168
:1009C00010E01DE019E045F008050FE045F01005C6
:1009D0000CE045F0200509E045F0400506E045F053
:1009E000800503E045F4807500E000BF00BF20688B
:1009F000806920F0700021688861042021684860C7
:100A00002DB1606A284360622046FFF71DFEBDE8F5
:100A1000F09F70B504460CB9012070BD94F8200019
:100A200010B9204600F0E4F82068006840F00100AA
:100A30002168086000F06EFC05460DE000F06AFCDD
:100A4000401B0A2808D9606A40F400306062052023
:100A500084F820000120E0E72068406800F00100F1
:100A60000028EBD02068006820F0020021680860B0
:100A700000F050FC05460DE000F04CFC401B0A283D
:100A800008D9606A40F400306062052084F82000D4
:100A90000120C2E72068406800F002000028EBD186
:100AA000207E012806D12068006840F0800021687F
:100AB000086005E02068006820F080002168086078
:100AC000607E012806D12068006840F0400021685F
:100AD000086005E02068006820F040002168086098
:100AE000A07E012806D12068006840F0200021681F
:100AF000086005E02068006820F020002168086098
:100B0000E07E012806D12068006820F010002168EE
:100B1000086005E02068006840F010002168086067
:100B2000207F012806D12068006840F00800216875
:100B3000086005E02068006820F00800216808606F
:100B4000607F012806D12068006840F00400216819
:100B5000086005E02068006820F004002168086053
:100B6000D4E90201084321690843616908436168C7
:100B7000491E08432168C86100206062012084F892
:100B80002000002049E710B50246002092F82030EE
:100B9000012B01D0022B07D11468A46804EA8164F8
:100BA000B4EB816F00D0012010BD000010B50446E9
:100BB0000C492068884213D10B48C06920F00070AE
:100BC0000949C8614FF44071084800F069F91320E1
:100BD00000F04AFD142000F047FD162000F044FD0F
:100BE00010BD00000064004000100240000C0140F5
:100BF00010B590B0044600200C900D900E900F9010
:100C00004049206888427AD100200790089001204E
:100C10000990002002900390049005900690012016
:100C20000A9002A93848FFF773FC02213648FFF703
:100C3000AFFB01213448FFF7ABFB4FF400713248A2
:100C4000FFF7A6FB4FF480612F48FFF7A1FB4FF49D
:100C500000412D48FFF79CFB00BF2C48C06940F0C5
:100C600000702A49C8610846C06900F00070019010
:100C700000BF00BF00BF0846806940F008008861DF
:100C80000846806900F00800019000BF00BF881589
:100C90000C9000200D900E900CA91D4800F09AF9C0
:100CA0004FF400700C9002200D9003200F900CA9BF
:100CB000174800F08FF900BF1649486820F4C0407B
:100CC00040F0E06040F48040486000BF00221146E0
:100CD000132000F0FBFC132000F0E8FC002211467A
:100CE000142000F0F3FC142000F0E0FC0022114678
:100CF000162000F0EBFC162000F0D8FC00BF10B06E
:100D000010BD00000064004070010020001002408F
:100D1000000C014000000140704770477047704769
:100D2000704770B5044694F82000022828D1206846
:100D3000006840F001002168086000F0EBFA054609
:100D40000DE000F0E7FA401B0A2808D9606A40F479
:100D500000306062052084F82000012070BD20680A
:100D6000406800F001000028EBD02068006820F007
:100D7000020021680860012084F820000020EDE7CF
:100D8000606A40F4801060620120E7E770477047B6
:100D9000704770477047704770470146002291F8CE
:100DA0002100022808D00420886300BF002081F8B9
:100DB000200000BF012070470868006820F00E0086
:100DC0000B6818600868006820F001000B68186064
:100DD00091F8403001209840CB6B5860012081F899
:100DE000210000BF002081F8200000BF1046E2E78C
:100DF00070B50446002594F82100022803D0042091
:100E0000A063012548E02068006820F00E002168FA
:100E100008602068006820F00100216808601F4910
:100E20002068884201D1012026E01C491431206845
:100E3000884201D110201FE01849283120688842DB
:100E400001D1801518E015493C312068884201D154
:100E5000801411E0114950312068884202D14FF4CA
:100E6000803009E00D4964312068884202D14FF496
:100E7000801001E04FF08070084908394860012077
:100E800084F8210000BF002084F8200000BF606BC0
:100E900010B12046616B8847284670BD08000240AB
:100EA0002DE9F04102460B4600207FE001278740F4
:100EB00007EA0301002978D0404F4FEA900C57F819
:100EC0002C4087074FEA177C0F2707FA0CF73C40A6
:100ED0003B4FBA4201D100270FE03A4FBA4201D14D
:100EE00001270AE0384FBA4201D1022705E0374F07
:100EF000BA4201D1032700E004274FEA807C4FEA81
:100F00001C7C07FA0CF7A74230D187074FEA177C01
:100F10000F2707FA0CF4294F4FEA900C57F82C7062
:100F2000A743DFF898C04FEA90084CF82870284F84
:100F30003F688F43DFF898C0CCF800700CF10407CD
:100F40003F688F430CF1040CCCF800700CF10407DF
:100F50003F688F430CF1040CCCF800700CF10407CF
:100F60003F688F430CF1040CCCF80070FF2901D8C6
:100F7000174600E0171D3D46FF2901D8870002E013
:100F8000A0F10807BF003E462F684FF00F0C0CFA87
:100F900006FC27EA0C074FF0040C0CFA06FC47EAA3
:100FA0000C072F60D7688F43D760401C23FA00F7E7
:100FB000002F7FF47BAFBDE8F08100000800014006
:100FC00000080140000C01400010014000140140E5
:100FD000000401402DE9F8470346002294466EE1E3
:100FE0004FF0010808FA02F4D1F8008008EA040082
:100FF000A0427DD1DFF8DCA2D1F80480A8EB0A0979
:10100000D0453AD014DCB8F1030F50D009DCB8F168
:10101000000F31D0B8F1010F1CD0B8F1020F49D147
:1010200020E0B8F1110F18D0B8F1120F42D11EE034
:10103000B9F5881F25D006DCB9F5803F20D0B9F579
:10104000801F37D11AE0B9F5001F18D0B9F5041F79
:1010500030D117E0D1F80CC02DE0D1F80C8008F1A8
:10106000040C28E0D1F80C8008F1080C23E0D1F83A
:101070000C8008F10C0C1EE000BF00BF00BF00BFD9
:1010800000BF00BFD1F80880B8F1000F02D14FF0C7
:10109000040C0BE0D1F80880B8F1010F03D14FF038
:1010A000080C1C6102E04FF0080C5C6103E04FF09B
:1010B000000C00E000BF00BFFF2801D8984601E007
:1010C00003F104084646FF2802D84FEA820803E0ED
:1010D000A2F108084FEA88084746D6F800804FF08A
:1010E0000F0909FA07F928EA09080CFA07F900E0DC
:1010F00088E048EA0908C6F80080D1F8048008F0C2
:101100008058B8F1805F7DD100BFDFF8CC81D8F87E
:10111000188048F00108DFF8C091C9F81880C84667
:10112000D8F8188008F00108CDF8008000BF00BF93
:101130004FEAB9384FEA920958F829504FEA8278B5
:101140004FEA18794FF00F0808FA09F825EA080560
:10115000DFF88881434502D14FF0000816E0DFF840
:101160008081434502D14FF001080FE0DFF8748120
:10117000434502D14FF0020808E0DFF86C81434597
:1011800002D14FF0030801E04FF004084FEA8279E2
:101190004FEA197908FA09F848EA0505DFF84C81A1
:1011A0004FEA920948F82950D1F8048008F48038B1
:1011B000B8F5803F0AD1DFF83881D8F8008048EAD6
:1011C0000008DFF82C91C9F8008009E0DFF82081E1
:1011D000D8F8008028EA0008DFF81491C9F80080E8
:1011E000D1F8048008F40038B8F5003F10D1DFF8DA
:1011F000008108F10408D8F8008048EA0008DFF808
:10120000F09000E05AE009F10409C9F800800DE00F
:10121000DFF8DC8008F10408D8F8008028EA00082C
:10122000DFF8CC9009F10409C9F80080D1F80480F6
:1012300008F48018B8F5801F0ED1DFF8B48008F1EB
:101240000808D8F8008048EA0008DFF8A49009F1FF
:101250000809C9F800800DE0DFF8948008F108085B
:10126000D8F8008028EA0008DFF8849009F108091E
:10127000C9F80080D1F8048008F40018B8F5001F00
:101280000ED1DFF86C8008F10C08D8F8008048EA2D
:101290000008DFF85C9009F10C09C9F800800DE046
:1012A000DFF84C8008F10C08D8F8008028EA000824
:1012B000DFF83C9009F10C09C9F80080521CD1F804
:1012C000008028FA02F8B8F1000F7FF489AEBDE87B
:1012D000F8870000000011100010024000080140D3
:1012E000000C0140001001400014014008000140C2
:1012F0000004014010B5C26821EA020302EA0104B9
:1013000043EA0443036110BD0AB1016101E00B042B
:101310000361704701480068704700000C0000201E
:1013200070B504460CB9012070BD94F83D0028B991
:10133000002084F83C00204600F0DAF8242084F8ED
:101340003D002068006820F00100216808602068E6
:10135000006840F40040216808602068006820F4BC
:1013600000402168086000F0CFFA05465C496068DB
:10137000884206D85B48854201D2012007E0002060
:1013800005E05948854201D2012000E000200128F3
:1013900000D1C9E75548B5FBF0F62068406820F059
:1013A0003F003043216848604D496068884201D859
:1013B000701C07E04FF4967070434FF47A71B0FBE5
:1013C000F1F0401C2168096A21F03F0108432168BF
:1013D000086243496068884214D8681E6168490001
:1013E000B0FBF1F0401CC0F30B00042801D2042034
:1013F0003DE0681E61684900B0FBF1F0401CC0F39D
:101400000B0034E0A06838B9681E616801EB410147
:10141000B0FBF1F0401C0AE0681E616801EBC102FC
:1014200002EB0111B0FBF1F0401C40F48040C0F32E
:101430000B0008B901201AE0A06848B9681E61686D
:1014400001EB4101B0FBF1F0401CC0F30B000CE0DC
:10145000681E616801EBC10202EB0111B0FBF1F003
:10146000401CC0F30B0040F4804040F40040216871
:10147000C9694CF6FF72914308432168C861D4E9F9
:10148000070108432168096821F0C0010843216869
:101490000860D4E9031008432168896848F2FF32E4
:1014A0009143084321688860D4E905010843216815
:1014B000C96821F0FF0108432168C86020680068FE
:1014C00040F001002168086000202064202084F89A
:1014D0003D000020206384F83E0000BF24E70000A8
:1014E000A086010080841E0000093D0040420F00DC
:1014F00010B586B004460020029003900490059039
:1015000015492068884225D100BF1448806940F001
:101510000800124988610846806900F008000190BF
:1015200000BF00BFC020029012200390032005904E
:1015300002A90B48FFF74EFD00BF0848C06940F400
:1015400000100649C8610846C06900F40010019007
:1015500000BF00BF06B010BD0054004000100240A4
:10156000000C014003480068034909780844014918
:10157000086070470C0000201400002010B50848D7
:10158000006840F0100006490860032000F0DCF815
:101590000F2000F007F800F02BF8002010BD00002D
:1015A0000020024070B504460E4800784FF47A716E
:1015B000B1FBF0F00C490968B1FBF0F5284600F0EA
:1015C0003FFC08B1012070BD102C07D2002221463B
:1015D000501E00F07BF80548046001E00120F2E7AE
:1015E0000020F0E714000020180000201000002068
:1015F00008B500BF1148806940F001000F498861BB
:101600000846806900F00100009000BF00BF00BFE5
:101610000846C06940F08050C8610846C06900F0C3
:101620008050009000BF00BF00BF0549486820F00F
:10163000E06040F00070486000BF08BD001002404C
:101640000000014010B501460846002807DB00F005
:101650001F0301229A40034B440943F8242000BF92
:1016600010BD000080E200E010B5014608460028E9
:1016700017DB00F01F0301229A400B4B440943F88B
:10168000242000BF00BF00BFBFF34F8F00BF00BFCB
:1016900000BF00BF00BF00BFBFF36F8F00BF00BF20
:1016A00000BF00BF10BD000080E100E00146084619
:1016B000002809DB00F01F0301229A4043099B0028
:1016C00003F1E023C3F8002100BF70472DE9F05F6C
:1016D00080460D461646002702F0BCF807463946FC
:1016E0002A46334601F00700C0F1070ABAF1040F99
:1016F00002D94FF0040A01E0C0F1070AD14600F117
:10170000040ABAF1070F02D24FF0000A01E0A0F17B
:10171000030AD4464FF0010A0AFA09FAAAF1010AAB
:101720000AEA020A0AFA0CFA4FF0010B0BFA0CFB58
:10173000ABF1010B0BEA030B4AEA0B0421464046CE
:1017400002F090F8BDE8F09F00BF00F00702064BE2
:1017500019684FF6FF031940044B0B4343EA02217B
:10176000014B196000BF70470CED00E00000FA0566
:1017700070B504460D460CB9012070BD5A4800688A
:1017800000F00700A8420ED25748006820F007007A
:101790002843554908600846006800F00700A84241
:1017A00001D00120E9E7207800F0020002281DD1D5
:1017B000207800F00400042805D14C48406840F42B
:1017C000E0604A494860207800F00800082805D108
:1017D0004648406840F46050444948604348406887
:1017E00020F0F000A168084340494860207800F0EC
:1017F000010078B36068012806D13C48006800F415
:10180000003090B90120B8E76068022806D1374857
:10181000006800F0007040B90120AEE7334800686E
:1018200000F0020008B90120A7E73048406820F026
:101830000300616808432D494860FFF76BFD0646C9
:1018400009E0FFF767FD801B41F28831884202D929
:10185000032092E707E02548406800F00C0061682B
:10186000B0EB810FEDD12048006800F00700A842DE
:101870000ED91D48006820F0070028431A49086067
:101880000846006800F00700A84201D0012074E774
:10189000207800F00400042807D11448406820F4A0
:1018A000E060E168084311494860207800F00800D2
:1018B000082808D10D48406820F46050216940EAAA
:1018C000C1000A49486000F03FF808494968C1F37F
:1018D0000311074A515CC840064908600648006881
:1018E000FFF760FE002048E70020024000100240A1
:1018F000C85B0008180000201000002001480068A4
:10190000704700001800002000B5FFF7F7FF0449FA
:101910004968C1F30221034A515CC84000BD000080
:1019200000100240D85B000800B5FFF7E7FF04494C
:101930004968C1F3C221034A515CC84000BD0000A0
:1019400000100240D85B0008F0B585B00FF26C0CB7
:101950009CE8E01001A8A0E8E0101CA52D68009507
:1019600000210022002300240020194D696801F0A5
:101970000C05F5B1042D02D0082D19D101E0154850
:1019800019E001ADC1F38346AC5D01F4803555B17A
:101990000F4D6D68C5F340451DF805200D4D65439D
:1019A000B5FBF2F302E00C4D04FB05F3184602E030
:1019B00000BF084800BF00BF05B0F0BD020304052A
:1019C000060708090A0B0C0D0E0F1010010200008B
:1019D0000010024000127A0000093D00F8B50446EC
:1019E0000CB90120F8BD207800F00100002878D063
:1019F000F848406800F00C0004280CD0F548406816
:101A000000F00C00082811D1F248406800F4803042
:101A1000B0F5803F0AD1EF48006800F4003000289C
:101A20005FD0606800285CD10120DBE700BF606800
:101A3000B0F5803F06D1E748006840F48030E549C2
:101A4000086028E0606858B9E248006820F48030F7
:101A5000E04908600846006820F4802008601AE029
:101A60006068B0F5A02F0BD1DA48006840F4802000
:101A7000D84908600846006840F4803008600AE0F1
:101A8000D448006820F48030D249086008460068D5
:101A900020F48020086000BF606888B1FFF73AFC3E
:101AA000054606E0FFF736FC401B642801D90320F9
:101AB00098E7C848006800F400300028F2D010E031
:101AC000FFF728FC054606E0FFF724FC401B6428CE
:101AD00001D9032086E7BF48006800F400300028E1
:101AE000F2D1207800F00200022857D1B9484068AE
:101AF00000F00C0050B1B748406800F00C00082816
:101B000018D1B448406800F4803098B9B1480068F2
:101B100000F0020020B12069012801D0012061E716
:101B2000AC48006820F0F800616940EAC100A949AA
:101B3000086033E02069E8B10120A7490860FFF799
:101B4000E9FB054606E0FFF7E5FB401B022801D94B
:101B5000032047E79F48006800F002000028F2D009
:101B60009C48006820F0F800616940EAC10099498A
:101B7000086013E0002098490860FFF7CBFB05469A
:101B800006E0FFF7C7FB401B022801D9032029E725
:101B90009048006800F002000028F2D1207800F0A0
:101BA000080008282DD1A069B8B101208B49086030
:101BB000FFF7B0FB054606E0FFF7ACFB401B022831
:101BC00001D903200EE78348406A00F00200002894
:101BD000F2D0012001F0AEF913E000207F49086047
:101BE000FFF798FB054606E0FFF794FB401B022831
:101BF00001D90320F6E67748406A00F00200002889
:101C0000F2D1207800F00400042873D10027714835
:101C1000C06900F0805070B900BF6E48C06940F0E4
:101C200080506C49C8610846C06900F0805000903F
:101C300000BF00BF01276A48006800F48070B0B997
:101C40006748006840F4807065490860FFF762FBF0
:101C5000054606E0FFF75EFB401B642801D9032020
:101C6000C0E65F48006800F480700028F2D000BF32
:101C7000E068012806D15748006A40F00100554944
:101C8000086227E0E06858B95248006A20F0010075
:101C9000504908620846006A20F00400086219E012
:101CA000E06805280BD14B48006A40F00400494920
:101CB00008620846006A40F0010008620AE04548F0
:101CC000006A20F00100434908620846006A20F0DB
:101CD0000400086200BFE068A0B1FFF71BFB0546E7
:101CE00009E0FFF717FB401B41F28831884202D917
:101CF000032077E622E03748006A00F0020000285F
:101D0000EFD012E0FFF706FB054608E0FFF702FB05
:101D1000401B41F28831884201D9032062E62D48F8
:101D2000006A00F002000028F0D1012F05D12948F7
:101D3000C06920F080502749C86100BFE069C8B37E
:101D40002448406800F00C00082860D0E0690228B0
:101D500048D1002020490866FFF7DCFA054606E076
:101D6000FFF7D8FA401B022801D903203AE61948A8
:101D7000006800F000700028F2D1206AB0F5803FC2
:101D800007D11448406820F40030A1680843114985
:101D90004860D4E9080108430E49496821F47411E8
:101DA00008430C49486001200B490866FFF7B2FA66
:101DB000054607E03DE0FFF7ADFA401B022801D9D8
:101DC00003200FE60348006800F000700028F2D0FE
:101DD0002FE0000000100240000042428004424216
:101DE00000700040002014490866FFF793FA05468A
:101DF00006E0FFF78FFA401B022801D90320F1E526
:101E00000E48006800F000700028F2D111E0E0698F
:101E1000012800D1E6E50948466806F48031206AC9
:101E2000814204D106F47011606A814201D0012020
:101E3000D8E50020D6E50000000042420010024034
:101E400070B504462546681EB0F1807F01D301209D
:101E50000FE0681E4FF0E02148610F214FF0FF3086
:101E600001F000FD00204FF0E021886107200861AB
:101E7000002070BD7047704730B502460B4600BF6A
:101E800092F83C00012801D1022030BD012082F8E7
:101E90003C0000BF022082F83D00106844681068D2
:101EA000816824F070041868044310684460104D81
:101EB0001068A8420BD01068B0F1804F07D00D4DCC
:101EC0001068A84203D00C4D1068A84205D121F03B
:101ED00080015868014310688160012082F83D004C
:101EE00000BF002082F83C0000BF00BFCDE700002B
:101EF000002C0140000400400008004010B50446DA
:101F00000CB9012010BD94F83D0028B9002084F8D8
:101F10003C00204600F026F8022084F83D00211DF8
:101F2000206801F0FDF8012084F8460000BF84F825
:101F30003E0001213F20015540200155412001551F
:101F400000BF00BF012084F8420043200155442017
:101F500001554520015500BF012084F83D000020B7
:101F6000D0E7000038B504460D492068884215D1F5
:101F700000BF0C48C06940F004000A49C861084627
:101F8000C06900F00400009000BF00BF00221146AD
:101F90001E20FFF79BFB1E20FFF788FB38BD0000CB
:101FA00000080040001002402DE9F04104460D46B3
:101FB00000BF94F83C00012802D10220BDE8F08166
:101FC000012084F83C0000BF022084F83D00206816
:101FD000866826F0770626F47F46206886602868A3
:101FE000502833D00CDC202850D004DC00284BD003
:101FF000102851D149E0302849D040284CD139E04F
:1020000060282DD0702807D0B0F5805F03D0B0F5E0
:10201000005F41D10DE040E0D5E902136A68206815
:1020200001F0B8F82068866846F077062068866078
:1020300033E0D5E902136A68206801F0ABF8206844
:10204000806840F480402168886026E0EA6869681A
:10205000206801F0B3F85021206801F0A6F81CE0D8
:10206000EA686968206801F0BCF86021206801F026
:102070009CF812E0EA686968206801F09FF8402146
:10208000206801F092F808E000BF00BF00BF296897
:10209000206801F08AF800E000BF00BF012084F84A
:1020A0003D0000BF002084F83C0000BF00BF85E772
:1020B000704710B5044620680069C0F34000D8B1ED
:1020C0002068C068C0F34000B0B16FF00200216822
:1020D0000861012020772068806900F0030018B1B2
:1020E0002046FFF7E5FF05E0204600F0ADF820466A
:1020F00000F0ABF80020207720680069C0F3800072
:10210000D8B12068C068C0F38000B0B16FF004009F
:1021100021680861022020772068806900F44070FF
:1021200018B12046FFF7C4FF05E0204600F08CF808
:10213000204600F08AF80020207720680069C0F36C
:10214000C000D8B12068C068C0F3C000B0B16FF063
:10215000080021680861042020772068C06900F029
:10216000030018B12046FFF7A3FF05E0204600F06A
:102170006BF8204600F069F800202077206800699D
:10218000C0F30010D8B12068C068C0F30010B0B12F
:102190006FF0100021680861082020772068C0696E
:1021A00000F4407018B12046FFF782FF05E020469A
:1021B00000F04AF8204600F048F800202077206818
:1021C000006900F0010058B12068C06800F001000B
:1021D00030B16FF0010021680861204600F036F848
:1021E00020680069C0F3C01058B12068C068C0F30F
:1021F000C01030B16FF08000216808612046FFF701
:1022000039FE20680069C0F3801058B12068C068AA
:10221000C0F3801030B16FF04000216808612046A3
:1022200000F019F820680069C0F3401058B1206828
:10223000C068C0F3401030B16FF020002168086121
:102240002046FFF718FE10BD7047704710B50446D2
:1022500003F094F910BD70477047704701460022A3
:10226000002391F83D2091F83E3042EA0300704788
:102270002DE9F84F0446206805682068C668206884
:1022800047694FF00009CA4605F00F09B9F1000F80
:102290000AD105F0200038B106F0200020B1204618
:1022A00001F0ADF8BDE8F88FB9F1000F71D007F07B
:1022B000010018B906F4907000286AD005F00100FA
:1022C00030B106F4807018B1206C40F00100206439
:1022D00005F0040030B107F0010018B1206C40F0A7
:1022E0000200206405F0020030B107F0010018B1CF
:1022F000206C40F00400206405F0080048B106F0AE
:10230000200010B907F0010018B1206C40F008005F
:102310002064206C68B305F0200028B106F020008E
:1023200010B1204601F06BF820684069C0F3801AB4
:10233000206C00F0080010B9BAF1000F22D020463E
:1023400001F032F82068406900F04000B0B1206828
:10235000406920F0400021684861A06B50B15648A8
:10236000A16B4863A06BFEF743FD10B1A06B416BFE
:1023700088470CE02046FFF770FF08E02046FFF793
:102380006CFF04E02046FFF768FF0020206489E727
:10239000FFE7206B012878D105F01000002874D0E9
:1023A00006F01000002870D000BF002000902068C8
:1023B0000068009020684068009000BF00BF20685F
:1023C000406900F04000C0B3A06B006840681FFA8D
:1023D00080F8B8F1000F2FD0A08D40452CDDA4F877
:1023E0002E80A06B806920281FD02068C06820F450
:1023F00080702168C8602068406920F00100216871
:1024000048612068406920F0400021684861202030
:1024100084F83E00002020632068C06820F010008F
:102420002168C860A06BFEF7B8FCA08DE28D801A11
:1024300081B22046FFF710FF34E7FFE7A08DE18D62
:10244000401A1FFA80F8E08DE8B1B8F1000F1AD0F9
:102450002068C06820F490702168C86020684069D6
:1024600020F0010021684861202084F83E0000200F
:1024700020632068C06820F010002168C8604146D1
:102480002046FFF7E9FE0DE7FFE705F0800030B1D9
:1024900006F0800018B1204601F0C5F802E705F00B
:1024A000400030B106F0400018B1204600F097FF20
:1024B000F8E600BFF6E600009533000810B50446C4
:1024C0000CB9012010BDA06900B100E000BF94F874
:1024D0003D0028B9002084F83C00204600F028F890
:1024E000242084F83D002068C06820F40050216852
:1024F000C860204600F0F6FF2068006920F4904094
:10250000216808612068406920F02A00216848613C
:102510002068C06840F400502168C8600020206432
:10252000202084F83D0084F83E000020CAE7000027
:1025300010B586B0044600200290039004900590E8
:1025400055492068884237D100BF5448806940F41B
:102550008040524988610846806900F480400190BB
:1025600000BF00BF00BF0846806940F004008861DA
:102570000846806900F00400019000BF00BF4815C4
:102580000290022003900320059002A94448FEF720
:1025900021FD4FF48060029000200390049002A976
:1025A0003F48FEF717FD002211462520FFF78EF861
:1025B0002520FFF77BF86DE03A49206888422ED14C
:1025C00000BF3648C06940F400303449C86108464D
:1025D000C06900F40030019000BF00BF00BF084692
:1025E000806940F0040088610846806900F00400BA
:1025F000019000BF00BF042002900220039003203E
:10260000059002A92648FEF7E5FC0820029000206C
:102610000390049002A92248FEF7DCFC3AE022492C
:102620002068884236D100BF1C48C06940F4802031
:102630001A49C8610846C06900F48020019000BFB3
:1026400000BF00BF0846806940F008008861084666
:10265000806900F00800019000BF00BF08150290DB
:10266000022003900320059002A91048FEF7B2FC57
:102670004FF40060029000200390049002A90B48E0
:10268000FEF7A8FC002211462720FFF71FF827209D
:10269000FFF70CF806B010BD0038014000100240F2
:1026A000000801400044004000480040000C014088
:1026B0002DE9F84F04460E46174699464FF0000A9A
:1026C00094F83E0020285FD106B117B90120BDE87B
:1026D000F88F00BF94F83C00012801D10220F6E7F2
:1026E000012084F83C0000BF00202064222084F8F0
:1026F0003E0000202063FEF70DFE8246A785E78599
:10270000A068B0F5805F04D1206910B90025B046FB
:1027100002E035464FF0000800BF002084F83C007E
:1027200000BF29E05346002220212046CDF800902A
:1027300000F0A9FF08B10320C9E745B92068406847
:10274000C0F30800A8F8000008F1020811E0A06832
:10275000B0F5805F03D0A06828B9206918B9206857
:102760004068287004E02068406800F07F0028700E
:102770006D1CE08D401EE085E08D0028D2D1202028
:1027800084F83E000020A2E70220A0E770B50446CE
:102790000D46164694F83E00202816D105B10EB914
:1027A000012070BD00BF94F83C00012801D1022037
:1027B000F7E7012084F83C0000BF00202063324688
:1027C0002946204600F00CFFEBE70220E9E7000075
:1027D0001D4A0168914236D11C49098801F4004123
:1027E00089BB1A49098801F4804171B118490978F7
:1027F0000A2903D00021154A118024E013490988D1
:1028000041F40041114A11801DE0114909780D2958
:1028100006D10E49098841F480410C4A118012E02A
:102820000B490978094A1288C2F30D02094B9954E1
:1028300006490988491C054A118011460988C7299B
:1028400001DD0021118070470038014004000020A4
:1028500006000020000300202DE9F84F04460E4634
:10286000174699464FF0000A94F83D0020285AD1A7
:1028700006B117B90120BDE8F88F00BF94F83C00FD
:10288000012801D10220F6E7012084F83C0000BFB6
:1028900000202064212084F83D00FEF73BFD8246A5
:1028A000A784E784A068B0F5805F04D1206910B9DF
:1028B0000025B04602E035464FF0000800BF00207A
:1028C00084F83C0000BF1BE05346002280212046D4
:1028D000CDF8009000F0D7FE08B10320CBE745B952
:1028E000B8F80000C0F308002168486008F1020849
:1028F00003E02878216848606D1CE08C401EE0846D
:10290000E08C0028E0D15346002240212046CDF83B
:10291000009000F0B8FE08B10320ACE7202084F856
:102920003D000020A7E70220A5E7704700BFFEE7B3
:1029300070B50446002500BF00259120005D0628E3
:102940001ED2DFE800F0031E4C4D5C7094F854007A
:10295000032815DB04F1700002F028FE80B904F1B1
:10296000940104F1700002F041FE40B10121912078
:102970000155002084F890000021AC20015501256C
:1029800067E094F8993094221159207804F19A0262
:10299000A668B04784F8980094F89000401C84F82A
:1029A000900094F89800FF280ED002219120015544
:1029B0000021AC200155012594F8540081280DD147
:1029C000032084F8540009E094F8901094F844002F
:1029D000814203DB042191200155012539E038E0D3
:1029E00094F8901094F84400814203DB0421912074
:1029F000015502E0012191200155012529E0002126
:102A000091200155D4F8A80020B10121D4E9290270
:102A1000904706E0206D20B10121226DD4F8A4007A
:102A20009047012515E0002191200155D4F8A80018
:102A300028B10220D4E9292101F068FA07E0206DCD
:102A400028B10220D4F8A420216D01F05FFA0125FD
:102A500000BF00BF012D04D19120005D04287FF448
:102A60006BAF25B122780421012001F04FFA70BD2F
:102A700010B504469120005D022811D194F8901001
:102A800094F84400814203DB04219120015502E0C7
:102A900003219120015522780421012001F036FA0A
:102AA00010BD70B504460D469120005D022803D08C
:102AB0009120005D03280DD194F89800A84209D117
:102AC00005219120015594F85400032802DB20468B
:102AD000FFF72EFF70BD000010B5002414E004EBDA
:102AE000440101EBC4010F4A02EB0110B021FDF7D4
:102AF00032FBFF2004EB440101EBC401094A02EB65
:102B000001110870601CC4B2022CE8D300F090FAE6
:102B10000549012001F014FA0449022001F010FADD
:102B200010BD0000900400202903000811030008D4
:102B300010B524210E48FDF70EFB14210D48FDF7BA
:102B40000AFB0D4800F00AFA044624B1142221467B
:102B50000848FDF7E7FA0848203000F0FFF904467E
:102B60002CB11422214603481430FDF7DBFA10BDC6
:102B70006C04002058040020EC5B00082DE9F041B3
:102B800080460D46164600244046FDF7DBFB044612
:102B90000CB105B116B90020BDE8F081287818B154
:102BA00094F85400012801D00020F5E795F82000A2
:102BB00000F0010018B1A86A08B90020ECE795F808
:102BC000251084F8451094F8450010B9322184F896
:102BD000451094F8451001EB4101C80002F028FBB4
:102BE000C4F88C00D4F88C0048B194F84530182211
:102BF00004F17000D4F88C1002F0EAFC01E000202F
:102C0000CAE795F8200000F00100D8B994F8451003
:102C1000080102F00DFBC4F88800D4F8880048B120
:102C200094F84530102204F15800D4F8881002F0CE
:102C3000CFFC07E0D4F88C0002F03CF90020C4F887
:102C40008C00A9E7296A216404F120072021384675
:102C5000FDF781FA1F2229463846FDF763FAE86A34
:102C6000F862A86AB86295F8240087F82400286BF7
:102C70003863084830610848F0600848B060084888
:102C800070600848306008487061022084F8540081
:102C9000012081E7555500088153000801540008C0
:102CA0001B540008A55400089D52000810B50F4899
:102CB0000F4908600920486000210D488160C1600B
:102CC0004FF4402101614FF48011416100210176F0
:102CD0000121417600218176C17601774177FDF7A8
:102CE00098FE08B1FDF72AFB10BD0000006400400B
:102CF0007001002000B585B0002001900290039083
:102D0000049000BF3148806940F020002F4988615D
:102D10000846806900F02000009000BF00BF00BF9F
:102D20000846806940F0040088610846806900F028
:102D30000400009000BF00BF00BF0846806940F05B
:102D4000080088610846806900F00800009000BF14
:102D500000BF002241F238011D48FEF7D5FA0022DB
:102D60004FF400411B48FEF7CFFA4FF4805001901A
:102D700001200290002003900220049001A9144831
:102D8000FEF728F94FF40040019001200290022044
:102D90000390049001A90F48FEF71CF90820019048
:102DA0000120029002200390049001A90848FEF738
:102DB00011F930200190012002900390022004902C
:102DC00001A90348FEF706F905B000BD0010024056
:102DD000000C01400008014010B50B480B49086089
:102DE0000B484860002109488160C1604FF4804170
:102DF0000161002141618161C1610162FEF790FAC8
:102E000008B1FDF79BFA10BD005400409801002066
:102E1000A086010000B587B00020039004900590C3
:102E200006900190029014481449086040F60F6023
:102E300048600021114881602321C16000210161A7
:102E40008161FFF75BF808B1FDF778FA4FF4805025
:102E5000039003A90948FFF7A7F808B1FDF76EFA38
:102E600000200190029001A90448FFF705F808B17D
:102E7000FDF764FA07B000BD00080040EC01002037
:102E800010B50B480B4908604FF4E1304860002151
:102E900008488160C16001610C21416100218161AC
:102EA000C161FFF70BFB08B1FDF748FA10BD000048
:102EB000003801403402002010B50B480B4908606F
:102EC0004FF4E1304860002108488160C160016131
:102ED0000C21416100218161C161FFF7EFFA08B166
:102EE000FDF72CFA10BD00000044004078020020DD
:102EF00010B50B480B4908604FF4E13048600021E1
:102F000008488160C16001610C214161002181613B
:102F1000C161FFF7D3FA08B1FDF710FA10BD000048
:102F200000480040BC02002000BFFEE700BFFEE7F3
:102F30007047000008B508490968C9084FF47A725B
:102F4000B1FBF2F14143009100BF00BF00994A1E5E
:102F500000920029F9D108BD1800002070B505467F
:102F60001DB1686808B1A86808B9002070BD0024C8
:102F70000EE004EB440000EBC4001B4901EB001021
:102F800000782978884201D10020EFE7601CC4B2A4
:102F9000022CEED3002422E004EB440000EBC4003A
:102FA000114901EB00100078FF2816D104EB440111
:102FB00001EBC4010C4A02EB011020222946FDF767
:102FC000B1F8012004EB440101EBC401064A02EB15
:102FD000011181F854000548C8E7601CC4B2022CF6
:102FE000DAD30020C2E70000900400207000002027
:102FF00070470000044801680068401C024A1060E5
:1030000001B972B6704700001C0000200748006834
:10301000012804D100200549086062B604E0034895
:103020000068401E01490860704700001C00002035
:1030300010B50948006820B9084800F0F9FF0649B2
:1030400008600548006801F086F820B90A210248A6
:10305000006801F073F810BD84000020D557000807
:1030600010B50E480068401C0C490860084600680E
:103070004FF47A71B0FBF1F201FB1200012804D188
:1030800007480068401C064908600648007810B9E7
:10309000012004490870FEF765FA10BD20000020E9
:1030A000080000202400002000B58FB0282105A8CA
:1030B000FDF751F814216846FDF74DF80120059001
:1030C00000040690002007900120099002200C9037
:1030D000C1030D914FF4E0110E9105A8FEF77EFC9F
:1030E00008B1FDF72BF90F2000900220019000207D
:1030F00002904FF480600390002004900221684603
:10310000FEF736FB08B1FDF719F90FB000BD7047A7
:1031100010B50248FEF7CDFF10BD0000EC01002005
:1031200010B50268184B984208D0B0F1804F05D016
:10313000164B984202D0164B984203D122F07002EF
:103140004B681A43104B984208D0B0F1804F05D01D
:103150000E4B984202D00E4B984203D122F440729B
:10316000CB681A4322F080034C6943EA04020260F0
:103170008B68C3620B688362034B984201D10B6971
:1031800003630123436110BD002C01400004004093
:103190000008004030B50C46816821F47F4142EAC6
:1031A000032525432943816030BD0A46816821F00B
:1031B000700142F0070319438160704730B50B4638
:1031C0001446026A056A25F001050562816921F04D
:1031D000F00141EA041122F00A021A4381610262FD
:1031E00030BD30B50B461446056A25F01005056262
:1031F0008169026A21F4704141EA043122F0A0029F
:1032000042EA03128161026230BD000002460023DF
:1032100021B90D4800681060012070470A48036812
:103220001068984205D81068181A884209D30120FE
:10323000F3E71068C0F1FF301844884201D3012041
:10324000EBE70020E9E70000200000204F4800786D
:1032500001280AD14E48C068401C4D49C860012071
:10326000087000204949087000E070474848C0686D
:103270000521B0FBF1F201FB120030B94448C068EF
:1032800018B101204249487000E0EEE74048C068AC
:103290000A21B0FBF1F201FB120028B93C48C068DA
:1032A00010B101203A4988703948C0681421B0FB38
:1032B000F1F201FB120028B93548C06810B10120B5
:1032C0003349C8703248C0683221B0FBF1F201FBCB
:1032D000120028B92E48C06810B101202C4908718D
:1032E0002B48C0686421B0FBF1F201FB120028B941
:1032F0002748C06810B10120254948712448C0689A
:103300004FF4FA71B0FBF1F201FB120028B920482A
:10331000C06810B101201E4988711D48C0684FF473
:103320007A71B0FBF1F201FB120028B91848C068AD
:1033300010B101201649C8711548C06840F2DC512F
:10334000B0FBF1F201FB120028B91148C06810B1BE
:1033500001200F4908720E48C0684FF4FA61B0FBB3
:10336000F1F201FB120028B90948C06810B1012030
:10337000074948720648C06841F27071884202D31A
:1033800000200349C86000BF6FE700002400002050
:103390000C04002070B505466C6A0020E085E084CE
:1033A0002046FEF75AFF70BD0168C96821F490718C
:1033B0000268D1600168496921F001010268516128
:1033C000016B012905D10168C96821F0100102686B
:1033D000D160202180F83E1000210163704710B5B4
:1033E00004462068C06820F040002168C8602020A2
:1033F00084F83D002046FFF798FA002010BDF8B58C
:10340000044694F83E00222869D1A068B0F5805F98
:103410000CD1206950B90025A66A20684068C0F325
:1034200008003080A06A801CA06215E0A56A002612
:10343000A068B0F5805F03D0A06828B9206918B9EA
:1034400020684068287004E02068406800F07F0031
:103450002870A06A401CA062E08D401E80B2E0850A
:10346000A8BB2068C06820F020002168C8602068E0
:10347000C06820F480702168C8602068406920F02E
:10348000010021684861202084F83E00206B01285B
:103490001ED1002020632068C06820F01000216841
:1034A000C8602068006800F0100010280AD100BF32
:1034B000002000902068006800902068406800901C
:1034C00000BF00BFA18D2046FEF7C6FE03E004E06A
:1034D0002046FFF77DF90020F8BD0020FCE7022020
:1034E000FAE7000070B504462168096921F44051EB
:1034F000E2681143226811612269A168114362697F
:1035000041EA02052168C96841F20C6291432943EE
:103510002268D1602168496921F44071A269114390
:10352000226851612D4A2168914202D1FEF7FCF9CF
:1035300001E0FEF7E9F900EBC00101EB0011626860
:103540009200B1FBF2F100EBC00202EB00126368E3
:103550009B00B2FBF3F26423B2FBF3F202EBC20373
:1035600003EB0212A1EB8201322202EB0111642271
:10357000B1FBF2F101F0F00100EBC00202EB00122E
:1035800063689B00B2FBF3F26423B2FBF3F201EB3E
:10359000021200EBC00101EB001163689B00B1FB5C
:1035A000F3F100EBC00303EB00136668B600B3FB56
:1035B000F6F36426B3FBF6F303EBC30606EB031343
:1035C000A1EB8301322303EB01116423B1FBF3F17F
:1035D00001F00F0111442268916070BD0038014074
:1035E00010B5034699629A85DA8500201864222076
:1035F00083F83E0000BF002083F83C0000BF18683D
:10360000C06840F480701C68E0601868406940F051
:1036100001001C6860611868C06840F020001C68E8
:10362000E060002010BD014691F83D00212828D11E
:103630008868B0F5805F0BD1086948B90A6A1088BC
:10364000C0F308000B685860086A801C086205E037
:103650000B6A581C086218780B685860C88C401EAA
:1036600080B2C88458B90868C06820F080000B6830
:10367000D8600868C06840F040000B68D86000203F
:1036800070470220FCE72DE9F04104460D4617463D
:103690009846069E21E0701CF8B12EB1FDF73AFE67
:1036A000A0EB0800B04218D92068C06820F4D070A0
:1036B0002168C8602068406920F0010021684861E5
:1036C000202084F83D0084F83E0000BF002084F8EC
:1036D0003C0000BF0320BDE8F0812068006828405E
:1036E000A84201D1012000E00020B842D3D0002040
:1036F000F1E7000010B500240C48FEF7B9FD00BF4B
:1037000001E0641C00BF0948FEF7A8FD2028F8D19D
:1037100000BF002401E0641C00BF012204490348EB
:10372000FFF734F80028F6D100BF10BDC803002011
:103730000600002010B50D48FEF79AFD0B48006802
:10374000C06800F0200008B101F020FF07480068C1
:10375000C06800F0800008B101F020FF2720FDF7CD
:1037600071FF0248FEF784FD10BD0000BC0200207E
:1037700010B501211748FDF706FAC4B244B10CB9DF
:10378000012000E0002002460021084600F00EFA69
:1037900002211048FDF7F7F9C4B244B10CB9012079
:1037A00000E0002002460121002000F0FFF9042182
:1037B0000848FDF7E8F9C4B244B10CB9012000E0B3
:1037C000002002460221002000F0F0F90148FCF739
:1037D000F9FF10BD7001002000B58FB006AB08AA3C
:1037E00000211248FCF731FFD0B9089801900998E0
:1037F00002900A98C0B28DF80C000B98C0B28DF8F8
:103800000D000C98C0B28DF80E0006A90DF10F0046
:103810000C9AFCF787FC01A9002000F07DF900BF9D
:103820000248FCF7CFFF0FB000BD00007001002080
:1038300000BFFEE70FB4054B10B503A9044A029878
:1038400000F034F810BC5DF814FB0000994E00083D
:103850000000002002480068C0F30220704700000A
:103860000CED00E010B5002804DB0A07130E054A32
:10387000135406E00A07140E034A00F00F031B1F3F
:10388000D45410BD00E400E018ED00E002E008C8E8
:10389000121F08C1002AFAD170477047002001E0CA
:1038A00001C1121F002AFBD1704700002DE9FF4F14
:1038B00089B09B460446002506E025280BD05A46D1
:1038C0000B999047641C6D1C20780028F5D10DB031
:1038D0002846BDE8F08F0027B8460122474900E09E
:1038E000074314F8013F203B02FA03F00842F7D1E6
:1038F00020782E2819D114F8010F47F004072A2840
:103900000ED06FF02F022078A0F1300109290CD8D9
:1039100008EB880102EB410100EB0108641CF2E7AF
:103920000A98641C50F8048B0A9020780028CED0A6
:10393000642808D0692806D075281ED05A460B99ED
:1039400090476D1C58E00A994FF00A0901C90A9185
:10395000002802DA40422D2102E0390504D52B214E
:103960008DF82010012103E0F90704D02021F7E7AA
:103970008A4608AE0DE00021FAE70A994FF00A09DD
:1039800001C90A91F7E74946FCF7F0FB303106F828
:10399000011D0028F7D1ADEB060000F120097807E2
:1039A00001D44FF00108C84502DDA8EB090000E092
:1039B00000208046002706E008A85A46C05D0B9903
:1039C00090476D1C7F1C5745F6DB04E030205A46BB
:1039D0000B9990476D1CB8F10001A8F10108F5DCC6
:1039E00005E016F8010B5A460B9990476D1CB9F18A
:1039F0000001A9F10109F4DC641C65E70928010054
:103A000010B58AB000F096FA0CE09DF8043002AAD6
:103A100005A80499FCF72EFC00208DF82700012052
:103A2000084908700848406840B1074801AB02AA3D
:103A300004A944680020A0470128E6D000F052F90C
:103A40000AB010BD6C0000201C04002010B5124804
:103A50000021016041608160C16018210F48FCF7BE
:103A60007AFB00F061FAFFF737F8FFF761F80B4ACD
:103A70000B490020FFF782F810B10AA0FFF7DAFE29
:103A80000648C06830B1054800231A461946C46884
:103A90001846A04710BD0000340400201C0400207C
:103AA0003800002063616E3120D0ADD2E9B3F5CA91
:103AB000BCBBAFB3C9B9A60D0A00000010B50446DF
:103AC00000200A4908600A48486004200872002063
:103AD000487201208872FF22082104480B30FCF74D
:103AE00033FB0248C47200F041FB10BD380D0020CA
:103AF000F456091010B504460648FDF712F908B14E
:103B0000002010BD0348FCF788FD08B10020F8E74D
:103B10000120F6E77001002070B505460C46012D26
:103B200000DB70BD05EB85000D4901EB80000069ED
:103B300088B1A37A207A042801D1606800E0206867
:103B4000014605EB8500064A02EB800004F10B02FA
:103B500006692846B047284600F092F900BFE0E722
:103B600058040020F0B587B007460C460E4E20687A
:103B7000019060680290207A0390607A0490A07AA5
:103B8000059000208DF818006B4604F10B0201A986
:103B90003046FCF712FC054615B1FF2007B0F0BD1A
:103BA0000098C0B2FAE700007001002070B504462A
:103BB0000D461646012C00DB70BD04EBC400144911
:103BC00001EB8000C0680121A9400840F0B104EB7E
:103BD000C4000F4901EB8000C0680121A94088435F
:103BE00004EBC4010A4A02EB8101C860204600F0E0
:103BF00047F904EB8400074951F8200030B104EB89
:103C0000840051F8202029462046904700BFD3E782
:103C10006C04002058040020024601207047000078
:103C200010B50446002004EBC401044A02EB8101F4
:103C300088602046FFF75EFF10BD00006C04002086
:103C400010B50446012C00DB10BD04EB84000D49C7
:103C500001EB8000806890B104EBC4000A4B03EBD9
:103C60008000C06808B1012000E00020014604EB9C
:103C70008400044B03EB800082682046904700BF1D
:103C8000E2E70000580400206C04002010B5044650
:103C9000012C00DB10BDFFF7ADF904EB84000F49E8
:103CA00001EB8000C06838B104EB84000A4602EBE7
:103CB0008000C16820468847FFF7A8F904EBC400DC
:103CC000074901EB8000C06830B1002004EBC4015B
:103CD000034A02EB8101C86000BFDBE75804002003
:103CE0006C0400207CB500200090019000246CE062
:103CF000374800EB0410007801284CD1344800EB21
:103D000004108089062807D2314800EB041080890E
:103D1000304931F8105001E02E4845892C4901EB1B
:103D20000411081D2946FFF771FA00284BD0FFF750
:103D300061F9274800EB04108089401C244901EBFD
:103D40000411888104EB4400234901EBC000C068E2
:103D500048B104EB440001EBC00000231A461946A9
:103D6000C6682046B0470220194901EB04110870CB
:103D700001208DF80000FFF749F9154901EB041106
:103D800001F108000021FFF741FA0120104901EB81
:103D90000411887317E00E4800EB04100078022825
:103DA00011D10B4901EB041101F108006721FFF764
:103DB0002DFA40B10020064901EB04118881044925
:103DC00001EB04110870601CC4B2012C90DB7CBDB7
:103DD00034040020E05B00081C0400202DE9F041C1
:103DE00004460D4616461F46012C02DB0020BDE8A6
:103DF000F081012004EBC401204A02EB81018860BC
:103E0000002004EBC40102EB8101487104EBC40003
:103E1000114601EB8000077104EBC40001EB800048
:103E2000C67004EBC40021F82050002004EBC4014C
:103E300002EB8101C86004EBC40002EB8001204664
:103E4000FFF7EAFE38B1022004EBC4010B4A02EB93
:103E50008101886006E0002004EBC401074A02EB00
:103E60008101886004EBC400044901EB8000806894
:103E7000022801D10120BAE70020B8E76C04002035
:103E8000012800DB704700BFFCE700002DE9F0418E
:103E900004460E4617469846012C07DA04EBC40088
:103EA000194901EB80008068022802D00020BDE89B
:103EB000F08104EBC401144A02EB810101F110000E
:103EC00043463A463146FCF7FCF904EBC4000E4A7F
:103ED00002EB800000F110012046FFF743FE05468B
:103EE000FF2D0ED004EBC400074901EB8000C16830
:103EF0000120A840014304EBC400034A02EB800008
:103F0000C1602846D3E700006C040020FEB50446DB
:103F10000D4616460094019502966946014801F047
:103F200082FBFEBD8008002010B500F0A9F800F06B
:103F300047F810BD10B500F055F800F0ABF810BD13
:103F400010B502460B4612B94FF0FF3010BD0021EC
:103F500014E01A4850F8310090420ED1174800EB97
:103F6000C1004360154800EBC100406818B900204B
:103F7000124C44F831000020E8E7491C1429E8D32A
:103F800013B94FF0FF30E1E7002111E00B4850F882
:103F9000310020B1094800EBC100406838B907483A
:103FA00040F8312000EBC10043600020CEE7491CFF
:103FB0001429EBD34FF0FF30C8E7000000060020C3
:103FC00010B54FF426710648FCF7C5F828230C22DB
:103FD0000349A03101F5F07001F0FAFA002010BD9C
:103FE000000600203EB518E069460F4801F0FEFAD1
:103FF00000240FE00D4850F834000099884208D1A1
:104000000A4800EBC400456815B19DE80700A847C1
:1040100002E0641C142CEDD300BF034801F0C6FA83
:104020000028E1D000203EBD8008002000060020CE
:1040300010B502460AB9002010BD002119E001EBBD
:1040400041000E4B03EB8000806880B901EB41001A
:1040500003EB80008260002001EB4103074C44F831
:10406000230001EB4100234603EB8000E4E7481CFA
:1040700081B21429E3D30020DEE700009808002075
:1040800010B5F0210248FCF766F8002010BD0000D2
:1040900098080020F8B5002700216846FFF7B6F819
:1040A0000098B84203D0781C0099814201D10020C9
:1040B000F8BD009F00243BE004EB44001E4901EBE7
:1040C0008000866804EB440051F820507DB376B33D
:1040D00004EB4401184A02EB8101081D2946FFF751
:1040E00095F8012823D104EB4400134901EB80002B
:1040F0008068A8B104EB440001EB8000406800999F
:10410000081AB0FBF5F004EB44010B4A02EB810105
:10411000496800FB051004EB440102EB8101486093
:104120002EB104EB4401044A02EB8100B047641C49
:10413000142CC1D30020BBE79808002070B50446BA
:104140000E46254605B970BD2E600021281DFFF7DB
:104150005DF800BFF7E701460A460AB9002070473C
:10416000106808B10120FAE70020F8E77CB50446A2
:10417000002611480068E0B10021207A042801D10E
:10418000606800E02068CDE90001607A08B9A07A93
:1041900000E000200346207A042801D1606800E096
:1041A00020680146044804F10B0205680020A84776
:1041B0007CBD0020FCE700001C04002070B5054613
:1041C0000C46064802880649681CFBF7ABFF03480B
:1041D0000088401C2080002070BD00008800002066
:1041E0008809002010B5002406480078012806D16F
:1041F00005480068804700200249087000E0062456
:10420000204610BD9F000020A40000202DE9F84F9B
:10421000054689464FF0000A01F088FC00B13EE0F7
:10422000B9F80000022838DB684601F073FA0098FC
:1042300040780602009880780643701C86B2009889
:10424000C078040200980079044304F0070038B1F4
:104250002046E11704EB5171C910491CCFB205E0AB
:104260002046E11704EB5171C1F3C707012C11DBA4
:104270006878B8420ED1002322463146A81C00F0CF
:1042800017FC8046B8F1000F09D0404601F065F9EF
:10429000824604E04FF0030A01E04FF0030A504663
:1042A000BDE8F88F2DE9F84F054689464FF0000A22
:1042B00001F03CFC00B13DE0B9F80000022837DB1A
:1042C000684601F027FA0098407806020098807846
:1042D0000643701C86B20098C078040200980079EA
:1042E000044304F0070038B12046E11704EB517194
:1042F000C910491CCFB205E02046E11704EB51710B
:10430000C1F3C707012C10DB6878B8420DD12246F3
:104310003146A81C00F06CFC8046B8F1000F09D0B3
:10432000404601F01AF9824604E04FF0030A01E02A
:104330004FF0030A5046BDE8F88F2DE9F8430546D3
:1043400088464FF0000901F0F1FB00B12CE0B8F80D
:104350000000022826DB684601F0DCF9009840786E
:104360000602009880780643701C86B20098C078D8
:104370000402009800790443012C10DB6000697886
:1043800088420CD1002322463146A81C00F09AFC3A
:1043900007464FB1384601F0E0F8814604E04FF09F
:1043A000030901E04FF003094846BDE8F8832DE911
:1043B000F843054688464FF0000901F0B7FB00B10D
:1043C0002BE0B8F80000022825DB684601F0A2F9CE
:1043D000009840780602009880780643701C86B2E8
:1043E0000098C0780402009800790443012C0FDB88
:1043F0006000697888420BD122463146A81C00F043
:10440000BDFC07464FB1384601F0A7F8814604E0ED
:104410004FF0030901E04FF003094846BDE8F88377
:104420002DE9F84F054689464FF0000B01F07EFB61
:1044300000B144E0B9F80000022840DB684601F012
:1044400069F9009840780602009880780643701C4D
:1044500086B20098C0780702009800790743009858
:1044600040794FEA00280098807940EA080808F16E
:1044700001001FFA80F80098C0794FEA002A0098DE
:10448000007A40EA0A0A78006978884215D1012347
:104490005246414600980A3000F014FC044634B9F4
:1044A00000233A463146A81C00F00CFC044634B107
:1044B000204601F052F8834601E04FF0030B5846C6
:1044C000BDE8F88F2DE9F84304460F464FF0000889
:1044D0003888052829D160780502A0780543681C32
:1044E00085B22079F0B9E078FF2801D0E078C8B92A
:1044F00000208DF80100E078FF2803D101208DF81D
:10450000000002E000208DF8000001231A46294631
:10451000684600F0CDFA06464EB1304601F01DF86F
:10452000804604E04FF0030801E04FF003084046E6
:10453000BDE8F8832DE9F04104460F464FF000082E
:104540003888052812D160780502A0780543681CD8
:1045500085B201231A462946E01C00F0B3FB06464B
:1045600036B1304600F0F9FF804601E04FF0030815
:104570004046BDE8F0812DE9F84F054689464FF0E9
:10458000000BB9F80000052803D001F0CFFA00288D
:1045900037D0684601F0BEF868780602A87806436E
:1045A000701C86B2E878040228790443009890F8D9
:1045B00005A004F0070038B12046E11704EB517163
:1045C000C910491CCFB205E02046E11704EB517138
:1045D000C1F3C707012C11DB57450FD10123224638
:1045E00031460098801D00F063FA8046B8F1000F54
:1045F00009D0404600F0B1FF834604E04FF0030BC2
:1046000001E04FF0030B5846BDE8F88F2DE9F84F55
:1046100082460F464FF000093888052802D001F085
:1046200085FA38B3684601F075F8009840780402BE
:10463000009880780443601C84B20098C07805021A
:10464000009800790543009890F80580680040457F
:104650000DD101232A4621460098801D00F032FB2F
:1046600006464EB1304600F078FF814604E04FF038
:10467000030901E04FF003094846BDE8F88F000048
:1046800001480078704700009E0000202DE9F041AD
:1046900004460D4616461F464FF00008F4B91A4866
:1046A0001A4908601A481B4908601B481B490860E2
:1046B0001B481C49086000201B4908601B481C4916
:1046C00008601C481C4908601C481D4908603A469F
:1046D0003146284600F03AF9804602E04FF00208E1
:1046E00000BF00BFB8F1000F0AD101F007F910B9FF
:1046F0004FF0030802E001201249087001F010F8A1
:104700004046BDE8F0810000854A0008A400002072
:10471000A14A0008A8000020F5490008A0000020D8
:104720009D490008AC000020B00000207559000829
:10473000B40000209D5A0008B8000020095A000863
:10474000BC0000209F0000202DE9F84F4FF000082A
:104750007548007830B174480078032802D00620EC
:10476000BDE8F88F684601F0A1F8012878D1BDF8BE
:10477000000004282AD004DC012807D0022870D1C8
:1047800008E008286ED01028F9D191E0032066498E
:104790000870C5E0654A66496648674B1B689847DC
:1047A000804600F05FFF0646B8F1000F07D1614870
:1047B0000078B04203D1042001F0A6F805E0012002
:1047C00000F0FCFF102001F09FF8A9E058480068B5
:1047D00000785A49087001205949087057480078F4
:1047E000C01120B152480068407808703FE00024B2
:1047F0003AE0544810F8340000B937E0514810F856
:1048000034004E49097888422DD1012000F0C4FFC0
:1048100001F08CF9B0B100F047FF44490880012550
:104820000DE0E8B200F0C4FF464800EBC4003F4989
:1048300042683F4800689047414908706D1C012D4F
:10484000EFDD09E03F4800EBC400384942683848D2
:10485000006890473A490870002000F09DFF05E08D
:104860005FE05CE012E0641C102CC2DB00BF344847
:10487000007830B1022000F0A1FF102001F044F8D0
:1048800003E000F017FF00F085FF49E0284800F042
:1048900041FF00F009FF814600F0E4FE82464A46EF
:1048A000234801685046284B1B689847804637E0EC
:1048B000FFF7E6FE07461E4800F02CFF27B1012F48
:1048C0000FD0022F27D119E000F0EEFE814600F054
:1048D000C9FE82464A4616480168504600F00EFF5F
:1048E00019E000F0E1FE814600F0BCFE82464A4637
:1048F0000F480168504600F0F5FE0CE000F0D4FED1
:10490000814600F0AFFE82464A460948016850469B
:1049100000F0DCFE00BF00BF00F03CFF00E000BF85
:1049200000BF00201CE700009F0000204E01002077
:10493000480100204C010020AC0000204D01002067
:1049400050010020C8000020A00000202DE9F04107
:1049500007460C4616464FF000083346082221460B
:10496000384600F0E9FF012802D04FF003080FE0BD
:10497000B4F5964F01D9232503E060000649B1FB49
:10498000F0F5A8B200F0F2FF012801D04FF00308C3
:104990004046BDE8F0810000A07F17002DE9F047F8
:1049A00004460D461646002710480088042810DBF0
:1049B0000E4801880E4800F05BFE50B90C480078A4
:1049C00020700A480088C01E30800948401C2860BA
:1049D00009E00648B0F800804FF004090188044857
:1049E00000F046FE82463846BDE8F087960000207B
:1049F000A50A00202DE9F04104460E4617464FF067
:104A00000008012C02DD0220BDE8F0811848007882
:104A1000012829D1701E1749086001201649088015
:104A20001448006804700846008838440880084626
:104A300001881048006800F01BFE05460E490888F2
:104A4000411C0D4B19800D490D542A121946088836
:104A5000411C198009490A540120094908700121A3
:104A6000002000F05FFE01E04FF005084046CBE774
:104A70008D0000209000002094000020A809002054
:104A80008C00002010B5002004490870002101208E
:104A900000F048FE00F079FE10BD00008D000020FF
:104AA00010B50021084600F03DFE00F068FE10BD84
:104AB0002DE9FF5F05460E4614469A4600200390F6
:104AC0002046E11704EB5171C910491C1FFA81F807
:104AD00000F0C8FD401E444901EBC00900200290CF
:104AE000402001904148008800904FF0010A701E5C
:104AF00086B20298864271DB3219DDE90110084462
:104B000082426BDC0099711A88B2C11700EB5171B7
:104B1000CF100099711A88B2C11700EB5171C910FA
:104B2000A0EBC1011FFA81FBBAF1000F03D0BAF16B
:104B3000010F51D126E00EE039467A1C97B201EB05
:104B400009000822594600F0FAFF05F8010BA8F108
:104B500001001FFA80F8B8F1000FEDDC6D1E204651
:104B6000E11704EB5171C910A4EBC1018CB2287894
:104B7000C4F10801884028702878C4F10801084170
:104B8000287029E00EE015F8013B39467A1C97B2EF
:104B900001EB09000822594600F0E6FFA8F10100E8
:104BA0001FFA80F8B8F1010FEDDC2046E11704EBA5
:104BB0005171C910A4EBC1018CB264B115F8013B6D
:104BC000E2B2394607F1010C1FFA8CF701EB09003C
:104BD000594600F0C9FF00BF02E0FFE70120039043
:104BE000039804B0BDE8F09F5C0100205A0100204A
:104BF0002DE9FE4F06460D46144600200290204641
:104C0000E11704EB5171C910491C1FFA81F900F03A
:104C100029FD401E294901EB400A4FF0000B1020EE
:104C20000190274800880090681E85B25D4540DBF2
:104C300029190198584481423BDC0099691A88B2CD
:104C4000C11700EB5171CF100099691A88B2C117D2
:104C500000EB5171C910A0EBC1011FFA81F80EE001
:104C600016F8013B39467A1C97B201EB0A0008227C
:104C7000414600F079FFA9F101001FFA80F9B9F16E
:104C8000010FEDDC2046E11704EB5171C910A4EBD4
:104C9000C1018CB27CB116F8013BE2B2394607F192
:104CA000010C1FFA8CF701EB0A00414600F05CFF93
:104CB00001E0012002900298BDE8FE8F580100201B
:104CC000560100202DE9FC5F04460F4616460020E1
:104CD000019000F0C7FC401E00EBC00101EB00108A
:104CE000244901EBC0084FF0000A4FF0640B224842
:104CF000008800904FF00109781E87B2574534DBD9
:104D0000B8190AEB0B0188422FDC0098381A85B2DB
:104D1000B9F1000F03D0B9F1010F25D110E00CE07B
:104D200038F81500001204F8010B18F8150004F803
:104D3000010B681C85B2701E86B2002EF0DC13E0F9
:104D40000FE014F8011B080228F8150014F8010BF5
:104D500038F81510084328F81500681C85B2701E35
:104D600086B2002EEDDC00BF01E001200190019829
:104D7000BDE8FC9F6E0C0020660100202DE9F84F75
:104D800004460D4617460020009000F06BFC401EC4
:104D900000EBC00101EB0010174901EBC0084FF018
:104DA00000094FF0640A1548B0F800B0681E85B2DB
:104DB0004D451BDBE81909EB0A01884216DCA5EB1F
:104DC0000B0086B20FE014F8011B080228F8160049
:104DD00014F8010B38F81610084328F81600701C58
:104DE00086B2781E87B2002FEDDC01E00120009032
:104DF0000098BDE8F88F0000A60B00206401002099
:104E00002DE9F84306460C4615461F464FF00008AC
:104E1000012E02DD4FF0020822E0384600F08CFE41
:104E200010B94FF005081BE0684600F073FC3046EF
:104E300000F0BEFC01200099087020120099487013
:104E400000998C7028120099C87000990D71052086
:104E500000F0BAFC082000F057FD00F005F880468D
:104E60004046BDE8F883000000200A49097820295F
:104E700007D0402906D0802906D0B1F5807F07D120
:104E800004E005E0042003E0032001E0062000BF69
:104E900000BF70475401002000BF054A126802F0AD
:104EA0004002002AF9D0C2B2014B1B1D1A607047A4
:104EB0000038014010B5002821D0114B0022001FFE
:104EC000196803E0814203D80A4649680029F9D1EC
:104ED00052B11368841A9C4204D1006818441060CF
:104EE000104602E0506000E0186039B102680B1A09
:104EF000934203D10B681A4402604968416010BDB7
:104F00006801002070B505460E463046FBF71AFAD8
:104F1000044604B970BD812D26D004DC042D07D0D1
:104F2000802D4DD116E0822D0AD0832D48D128E066
:104F300094F85400032802DB2046FDF7F9FC40E01A
:104F400094F85400032804DBE06C10B18220E16C7B
:104F5000884736E094F85400032804DBE06C10B175
:104F60008020E16C88472CE094F85400032807DB8C
:104F70002046FDF77DFDE06C10B18120E16C884793
:104F80001FE094F85400032819DB9120005D0228EB
:104F900006D104219120015522780120FEF7B6FFA9
:104FA000E06C18B18320E16C884708E0207800F0BD
:104FB00075F9207800231A46194600F0E1F900E05F
:104FC00000BF00BF00BFA5E770B506460D463046DE
:104FD000FBF7B8F904461CB394F85400022805DC2A
:104FE000E068E8B13046E168884719E094F8540079
:104FF000812808D13DB184F8540032468121012036
:10500000FEF784FF0CE094F85400812808D03DB9E5
:10501000802084F85400324680210120FEF776FF7C
:1050200070BD70B504460D4629462046FFF7CCFFFB
:1050300070BD70B505462846FBF784F904468CB16F
:1050400094F85400022805DCE06858B12846E1686D
:10505000884707E0832084F854002A4683210120F2
:10506000FEF754FF70BD00002DE9F04107460D46E4
:1050700090461E463846FBF765F90446002C39D0A9
:1050800094F85400032835DB94F85400802802D1AA
:10509000032084F8540094F8400000F0010038B177
:1050A000A06C38B3324641462846A36C984721E0AD
:1050B0001248056006710079002809DD0F48007963
:1050C000082805DC0D4802794146401DFBF72AF807
:1050D0000A4904F1580000F0A6FA04F1580000F063
:1050E0006EFA38B1822084F854003A4682210120B9
:1050F000FEF70CFF0120BDE8F0810000F005002064
:1051000070B506460C463046FBF71CF905461DB146
:10511000E1B22846FDF7C5FC70BD0000FCF72EFA91
:10512000FDF7C2FFFDF7E6FDFDF7C0FDFDF754FEFC
:10513000FDF7C2FEFDF7DCFEFDF7A2FEFDF76AFEFD
:1051400033A0FEF777FB00234FF4E132032118462A
:10515000FFF79CFAFFF746F8FEF778FC56E0FEF7FB
:1051600075F8FEF74DFC2E480078012803D1002089
:105170002B4908704AE02A484078012805D10020D0
:1051800027494870FFF7E0FA40E025488078012879
:1051900003D100202249887038E02148C0780128D6
:1051A00003D100201E49C87030E01D480079012855
:1051B00003D100201A49087128E0194840790128D4
:1051C00005D1002016494871FEF778FC1EE014480E
:1051D000807901280FD10020114988714FF4FA73AA
:1051E000012200211046FFF70BFE044621460DA0C8
:1051F000FEF720FB0AE00A48C079012806D100200A
:105200000749C87120210948FCF774F8A7E7000096
:1052100068656C6C6F20776F726C640D0A0000001B
:105220000C04002025640D0A00000000000C014061
:10523000F0B50B30154D20F007010024144A0FE0A3
:1052400003688B420BD38B4205D95E1A431847681B
:10525000C3E9006700E04368136002C004E0021D78
:1052600010680028ECD12046002802D1286808B137
:105270000020F0BD064A07481060074A121A22F0C3
:105280000702C0E9002401202860D7E76C01002054
:1052900068010020540D0020500F002070B5054615
:1052A0002846FBF74FF804461CB194F85400022836
:1052B00001DC002070BD022084F85400E06810B1C9
:1052C0002846E16888479120005D002834D0D4F852
:1052D000A800B0B19120005D052804D10021D4E9D7
:1052E0002902904728E09120005D042804D1012183
:1052F000D4E9290290471FE00321D4E9290290470D
:105300001AE0206DC0B19120005D052805D1002173
:10531000226DD4F8A40090470EE09120005D04288F
:1053200005D10121226DD4F8A400904704E00321A7
:10533000226DD4F8A400904715E004F1940104F123
:10534000700000F053F970B1D4F8A80020B1032127
:10535000D4E92902904706E0206D20B10321226D97
:10536000D4F8A400904704F1700000F01FF9002861
:10537000E3D0202104F19000FAF7EDFE012099E737
:105380002DE9F04105460E46174698462846FAF79D
:10539000D9FF04461CB194F85400012802DC002017
:1053A000BDE8F081606848B343463A463146284636
:1053B000D4F804C0E04708B3D4F88C0040B194F8A6
:1053C0004530182204F17000D4F88C1000F000F978
:1053D00094F8400000F0010058B9D4F8880040B1BA
:1053E00094F84530102204F15800D4F8881000F0E9
:1053F000EFF8032084F854000120D1E70020CFE724
:1054000070B5054600242846FAF79CFF044614B1FF
:1054100094F8540070BD0020FCE72DE9FF41804660
:105420000E4615461F464046FAF78CFF04464CB11F
:1054300094F85400022805DD25B194F8400000F0EE
:10544000010018B1002004B0BDE8F08104F158005B
:1054500000F0ACF808B10020F5E7694604F1580007
:1054600000F0C4F808B90020EDE7009830609DF81E
:10547000040038709DF8040000280ADD9DF804003F
:10548000082806DC9DF804200DF105012846FAF7EE
:1054900049FE94F85400822802D1032084F8540075
:1054A0000120D0E72DE9F04786B080460F4615462B
:1054B0001E46DDE90E9A00244046FAF743FF0446F3
:1054C00054B194F85400022806DD082E04DC04F1DF
:1054D000700000F074F818B1002006B0BDE8F08745
:1054E000FDF788FD94F85400832803D094F8540005
:1054F000032803DAFDF78AFD0020EEE7CDF814A0BB
:1055000000978DF80560CDF8109015B900208DF842
:1055100005009DF8050000280ADD9DF80500082813
:1055200006DC9DF8052029460DF10600FAF7FAFD84
:10553000FF208DF80400694604F1700000F073F854
:105540009120005D10B92046FDF7F2F9FDF75EFDF0
:105550000120C2E7034600207047014621B101291E
:1055600004D0072906D103E0002005E0022003E073
:10557000062001E0042000BF00BF704710B50248BC
:105580000068804710BD0000BC00002010B5024834
:105590000068804710BD0000B400002010B502482C
:1055A0000068804710BD0000B80000200146488810
:1055B00008B1886808B9012070470020FCE701465F
:1055C00048880A88904201DB012070470020FCE7F0
:1055D00010B50380002444808160828002FB0314A4
:1055E000C460846804618468446110BD70B5044679
:1055F0000D46608808B1A06808B9002070BDA28877
:1056000028466169FAF78EFDA188606908446061E7
:10561000E1686069884201D3A06860616088401ECB
:105620006080A088EAE770B504460D46608821884E
:10563000884201DAA06808B9002070BDA288294616
:105640002069FAF76FFDA188206908442061D4E938
:105650000310884201D3A06820616088401C6080EC
:105660000120EAE701480078704700009C00002014
:1056700070B502460C46FF25FF2309E012F8010B26
:1056800080EA03010648405C80EA05030548455C62
:10569000201EA4F10106B4B2F0D143EA052070BD8A
:1056A0002C5C00082C5D0008014800887047000051
:1056B0008E00002001200349087020200249088044
:1056C00070470000540100205201002010B5012352
:1056D000024C23701B02024C238010BD5401002099
:1056E0005201002010B50123024C23708023024C8C
:1056F000238010BD540100205201002010B5012369
:10570000024C23704023024C238010BD5401002022
:10571000520100200149016070470000A9090020E2
:105720007047000040B1124A1268D26842F020026D
:105730000F4B1B68DA6007E00D4A1268D26822F04E
:1057400020020B4B1B68DA6041B1094A1268D2682B
:1057500042F08002064B1B68DA6007E0044A1268D8
:10576000D26822F08002024B1B68DA6070470000AA
:10577000BC02002010B5022000F014F810BD7047E4
:1057800010B5012000F00EF810BD10B5002000F09B
:1057900009F810BD7047000001490870704700000B
:1057A0009D0000200149087070470000990000200A
:1057B00001490870704700009C00002001490870F2
:1057C000704700009E0000200149088070470000DB
:1057D0008E00002070B50546002462E004EB440012
:1057E00000EBC400304901EB001090F8540003288E
:1057F00000DA54E004EB440000EBC4002A4901EB5A
:10580000001090F8910001280AD104EB440000EB4D
:10581000C40001EB0010027804210120FEF776FBA2
:1058200004EB440000EBC4001F4901EB001090F8AA
:105830009100022832D104EB440000EBC40001EBDC
:10584000001090F8AC00401CC1B204EB440000EB27
:10585000C400154A02EB001080F8AC1004EB4400C1
:1058600000EBC400114601EB001090F8AC000228D8
:1058700014DB032104EB440000EBC40002EB001036
:1058800080F8911004EB440000EBC400114601EBDA
:105890000010027804210120FEF738FB00BF601CD5
:1058A000C4B2022C9ADB70BD9004002010B50446EF
:1058B00000F0AAF810480078042810D004DC012871
:1058C00007D0022814D107E008280BD010280FD1E8
:1058D0000BE0012020800BE00220208008E0042063
:1058E000208005E00820208002E01020208000BFFA
:1058F00000BF012010BD000054010020012001491B
:1059000008707047540100200146024A11700120BE
:10591000704700005401002010B5044601231A46C8
:1059200021460448FCF7C4FE08B1002010BD012048
:10593000FCE70000BC0200202DE9F04104460D46C2
:1059400016461F46FDF7D4FA0120BDE8F08100009D
:1059500001B501231A4669460348FCF77DFF08B1EB
:10596000002008BD0120FCE7BC0200200146012008
:105970007047000038B500246846FFF7CDFF1E4889
:10598000007830B101280AD002281DD003282FD179
:1059900002E0FFF7FAFE2BE0FFF7F7FE28E0FFF743
:1059A000EEFE002015490870154908809DF800207A
:1059B0000888411C124B198012490A5402200E49D2
:1059C0000870FFF7E2FE13E00D480088FF2809DCAD
:1059D0009DF800200A490888411C094B1980094993
:1059E0000A5402E0032004490870FFF7CEFE00BF0E
:1059F00000BF204638BD00008D0000208C00002034
:105A000096000020A50A002010B500241F48007849
:105A100020B1022807D0032812D109E00120FFF7A6
:105A200073FF04460DE00220FFF76EFF044608E016
:105A30000120FFF7C3FE1020FFF766FF044600E0D9
:105A400000BF00BF012011490870114800780228EA
:105A50000AD11048007830B90020FFF7AFFE1020BF
:105A6000FFF752FF044600E000BF00BF00200849D6
:105A70000870FFF784FE08480078022803D104204C
:105A8000FFF742FF0446204610BD00008D000020B5
:105A90008C000020980000209900002010B5002400
:105AA0001D48007810B1012831D104E00021012007
:105AB000FFF738FE2CE01948008878B118490968CA
:105AC0000878FFF745FF16480068401C1449086035
:105AD00012480088401E1149088017E011480078DC
:105AE00008B9012000E000200F49087000210120C2
:105AF000FFF718FE0220084908700B4800780128BB
:105B000002D1FFF737FE01E0FFF73AFE00E000BFE9
:105B100000BF204610BD00008C0000209400002033
:105B200090000020A809002098000020014800787B
:105B30007047000098000020014601207047F0B532
:105B400003460C461546E208A4EBC20087B20120CA
:105B5000A840401E86B2995C501C185C41EA0021A6
:105B600039413140C8B2F0BD2DE9F0430446154635
:105B70001F46C808A1EBC0081FFA88FC07FA0CF8FA
:105B80001FFA88F74FF0010808FA05F8A8F1010894
:105B90001FFA88F6A1EBC00806FA08F81FFA88F683
:105BA000225C00F1010814F8088042EA082222EA87
:105BB000060848EA070222544FEA222900F10108A8
:105BC00004F80890BDE8F083000000000000000029
:105BD0000102030406070809000000000102030493
:105BE0001E00C600C600C600C600C60000000000B9
:105BF000DD3D00088D3E0008213C0008000000004B
:105C00000000000000000000000000000100000093
:105C1000DD3D00088D3E0008213C0008000000002A
:105C200000000000000000000000000000C18140F2
:105C300001C0804101C0804100C1814001C080415C
:105C400000C1814000C1814001C0804101C080414C
:105C500000C1814000C1814001C0804100C181403C
:105C600001C0804101C0804100C1814001C080412C
:105C700000C1814000C1814001C0804100C181401C
:105C800001C0804101C0804100C1814000C181400C
:105C900001C0804101C0804100C1814001C08041FC
:105CA00000C1814000C1814001C0804101C08041EC
:105CB00000C1814000C1814001C0804100C18140DC
:105CC00001C0804101C0804100C1814000C18140CC
:105CD00001C0804101C0804100C1814001C08041BC
:105CE00000C1814000C1814001C0804100C18140AC
:105CF00001C0804101C0804100C1814001C080419C
:105D000000C1814000C1814001C0804101C080418B
:105D100000C1814000C1814001C0804100C181407B
:105D200001C0804101C0804100C1814000C0C1016B
:105D3000C30302C2C60607C705C5C404CC0C0DCDFB
:105D40000FCFCE0E0ACACB0BC90908C8D81819D96B
:105D50001BDBDA1A1EDEDF1FDD1D1CDC14D4D5159B
:105D6000D71716D6D21213D311D1D010F03031F18B
:105D700033F3F23236F6F737F53534F43CFCFD3DBB
:105D8000FF3F3EFEFA3A3BFB39F9F83828E8E929AB
:105D9000EB2B2AEAEE2E2FEF2DEDEC2CE42425E55B
:105DA00027E7E62622E2E323E12120E0A06061A1CB
:105DB00063A3A26266A6A767A56564A46CACAD6D7B
:105DC000AF6F6EAEAA6A6BAB69A9A86878B8B979EB
:105DD000BB7B7ABABE7E7FBF7DBDBC7CB47475B51B
:105DE00077B7B67672B2B373B17170B0509091510B
:105DF0009353529296565797559594549C5C5D9D3B
:105E00005F9F9E5E5A9A9B5B99595898884849892A
:105E10004B8B8A4A4E8E8F4F8D4D4C8C44848545DA
:105E20008747468682424383418180404C5E00081A
:105E30000000002070010000BC010008BC5E0008EA
:105E400070010020E01100009C38000801103210A1
:105E50004201031124F4A3E80300091CD5FBB3B5E8
:105E6000D0ADD2E90312030A1301511408C94F142B
:105E70000823501B0833041A6904011B022802324C
:105E80001113BD4133080413AF432A08AB1A3B0872
:105E900029D0130D4633080613354533081713214F
:105EA000442A08E4130D423308051AC510320F1AAC
:0C5EB000772029711AA518015800000085
:04000005080000ED02
:00000001FF
